:1000000009C018951895189518951895189518956C
:10001000189518958FE98DBFC0E9EFE84E2EDD27C2
:100020005D2EEEE3F0E0A0E6B0E088278D933197F7
:10003000E9F766248CE087BB8DEF88BBC298C39A32
:100040000027A6E38C9181FB0EF401E040E0041749
:1000500009F009C0C39882E390E013D1C39AE1E0AC
:10006000F0E000D1EDCF81E080936000009160006E
:10007000083010F009F02EC088B398E0892788BBBB
:1000800082E390E0FED088B398E0892788BB81E0C6
:100090008093610000916100063010F009F014C0F7
:1000A0000027A6E38C9181FB0EF401E040E00417E9
:1000B00009F001C0C3CF82E390E0E3D0A1E68C91C8
:1000C0008F5F8C9308F4E6CFA0E68C918F5F8C93C2
:1000D00008F4CCCF81E0809360000091600006308E
:1000E00010F009F027C088B398E0892788BB81E029
:1000F0008093610000916100043010F009F014C099
:100100000027A6E38C9181FB0EF401E040E0041788
:1001100009F001C093CF82E390E0B3D0A1E68C91C7
:100120008F5F8C9308F4E6CFA0E68C918F5F8C9361
:1001300008F4D3CFC3988AE090E0A3D00027A6E3C9
:100140008C9180FB0EF401E040E0041781E009F09F
:1001500080E08F930027A6E38C9184FB0EF401E0EE
:1001600040E0041781E009F080E09F918923882313
:1001700009F405C081E090E0A2E68D939C930027EE
:10018000A6E38C9180FB0EF401E041E0041781E0CE
:1001900009F080E08F930027A6E38C9184FB0EF496
:1001A00001E040E0041781E009F080E09F9189239D
:1001B000882309F405C082E090E0A2E68D939C9329
:1001C0000027A6E38C9180FB0EF401E040E00417C9
:1001D00081E009F080E08F930027A6E38C9184FBF7
:1001E0000EF401E041E0041781E009F080E09F9106
:1001F0008923882309F405C085E090E0A2E68D9369
:100200009C930027A6E38C9180FB0EF401E041E073
:10021000041781E009F080E08F930027A6E38C911A
:1002200084FB0EF401E041E0041781E009F080E076
:100230009F918923882309F405C08FE090E0A2E60E
:100240008D939C93C29AA2E68D919C911AD0C298EC
:1002500082E390E016D0C39AE6E0F0E003D0EECE61
:10026000F894FFCF88EE93E00CD03197D9F708953A
:100270003197F1F70895689462F80895E89462F868
:100280000895EF93FF93EE27E82BE92B31F0E0E69A
:10029000F9E03197F1F70197D1F7FF91EF910895C8
:00000001FF
